:020000040000FA
:1000000014288A010F3982074434313432343334AE
:100010003434353436343734383439343034453484
:100020004634413442344334831640308100D0306A
:100030008600003085008312850186019020CA2049
:1000400051218B01B301AE01AF012D20061C2528E3
:10005000442006182928B3142528B31C0800AF0B28
:100060000800AE0B0800AE01AF01B3101D215720F0
:10007000061FA420512108000230A200A301A30BF7
:100080003F28A20B3F280800B1018618B1150619B8
:1000900031158619B114061A311431088000840A0A
:1000A00004082C3A031D080024308400080058304E
:1000B00045065C21AD0134082406832050304406F7
:1000C0005C21350825068320443043065C21360830
:1000D00026068320393042065C2137082706832014
:1000E000543041065C2138082806832049304006F8
:1000F0005C213908290683203A082A0683203B0818
:100100002B068320080003198728AD010800AD0ADB
:100110002D082C0603198D280800013085060800DB
:100120008901343084009D208000840A0908123A35
:10013000031D93283C08AC00080083160814000037
:1001400083120808890A0800831289012408BB2049
:100150002508BB202608BB202708BB202808BB2079
:100160002908BB202A08BB202B08BB2024303202E0
:10017000BB209020080088008316081555308900A0
:10018000AA30890088148818C3280812081183121D
:10019000890A080085111E300F21F03086050330D2
:1001A0008604051505300F21051101300F210821A6
:1001B0000821F03086050230860408212830FB2013
:1001C0000630FB200F30FB200130FB2002300F21D6
:1001D000C830FB204930F9205430F9203930F9205B
:1001E0004430F9205030F9205830F92018214629A0
:1001F000303E8515FC288511B000F0308605300EA4
:100200000F3986040821F030860530080F3986043E
:10021000051501300F21051101300F210800A30041
:10022000A2010000A20B11290000A30B1129080054
:10023000FA300F21FA300F21080086128316D030D1
:10024000860083128030FB202030F9202030F920F6
:100250002030F9202030F9202030F9202030F920FA
:100260002030F9202030F9208030FB200408243A87
:1002700003194E210408B200243084000008012034
:10028000F920840A32080406031D3E298316DF3054
:100290008600831286162430840008002C308400E7
:1002A0000800243084008001840A04082C3A031DCD
:0E02B0005329243084000800031D252808006F
:02400E00F13F80
:10420000010002000300040005000600070008008A
:1042100005004200590020004900540039004400C4
:0442200050005800F2
:00000001FF
